:100000008601E130660085011030650038306200FD
:100010008B018C0107309F0083169F0183122030D3
:1000200084008001840A841F1128CC01CC14061C92
:10003000CC102E24033085008614302486108614BC
:1000400030248610861430248610023085004E2419
:1000500028303E240C303E2406303E245224861A9A
:100060003428061B342851282B242B2453304324B6
:1000700057304324493043245430432443304324ED
:10008000483043243D242B2445304324523043241C
:10009000523043244F304324523043242B242B240A
:1000A0002F2852242B2457304324413043244930F5
:1000B0004324543043241930B400FF303624B40BA9
:1000C0005D2852242B2443304324413043244C30B8
:1000D00043244930432442304324523043244130A6
:1000E00043243D2454304324493043244E30432498
:1000F0004730432490242830692406160930B40080
:10010000FF303624B40B8028902424306924383002
:100110007624061228305C24BB253830762424301F
:100120005C245F258A30BF007A30C000C101C20163
:100130002225243069243830762428305C24222576
:1001400038307624B230B8006630B9006030BA007A
:10015000B330BB005F252030692480303E24861AEE
:100160001029061B1029861F08294C08031DC528C5
:100170000230CC00C401C501C601C701CD01C801D0
:10018000C901CA01CB01CE0103294C08023C031D61
:10019000D6280130CC00C401C501C601C701CD017C
:1001A000C801C901CA01CB01CE0103294C08013C99
:1001B000031DE7280330CC00C401C501C601C701F7
:1001C000CD01C801C901CA01CB01CE0103294C08E8
:1001D000033C031DF8280730CC00C801C901CA013F
:1001E000CB01CE01C401C501C601C701CD01032960
:1001F000CC01C401C501C601C701CD01C801C901B7
:10020000CA01CB01CE01CC22861B04292E240F2942
:1002100090243208031D0F2928306924CC22CB2AD0
:10022000861E3129061F31292B242B2453304324C9
:10023000573043244930432454304324433043242B
:10024000483043243D242B2445304324523043245A
:10025000523043244F304324523043242B242B2448
:10026000CB2A861E152A90243208023C031D5729EA
:100270004E3043244F304324543043242B24413008
:1002800043244E3043242B24493043243D244E3014
:1002900043244430432455304324433043245430D2
:1002A00043244F304324523043242B24142A320851
:1002B000031D142A3830762428305C245F258130D1
:1002C000BF00C001C101C201BB2520307624222518
:1002D0002C3069242C3076248E30B8001C30B900C4
:1002E0004030BA00BB01BB25B91B89296F30BF0064
:1002F0002730C000C530C100AC30C200222581309B
:10030000BF00C001C101C201C3252C3076242225C3
:100310008B292C305C24861FA829443069242B2487
:100320002B242B244C3043247A3043243D30432467
:100330004C189E29B801B901BA01BB010A23483003
:100340004324793043244F08CD00861BA529142A65
:1003500044307624BB254C1C062A4408031DD829AA
:100360004508031DD8294608031DD8294708031D41
:10037000D829493043244E30432453304324453058
:10038000432452304324543043242B244C30432400
:100390003D247A3043242B24263043242B245A3006
:1003A000432445304324523043244F304324052A0C
:1003B0004C1DF429443076245F258730BF00483037
:1003C000C000C101C20122254C30432478304324AF
:1003D000253043244C3043247A3043243D30432499
:1003E0000A232B242B24052A4C3043247830432421
:1003F0002D3043244C3043247A3043243D30432471
:100400000A234830432479304324142A2B242B24F4
:100410002B244C304324783043243D3043240A239A
:100420004830432479304324CB2A90243830762432
:1004300028305C245F258130BF00C001C101C201AA
:10044000BB25B91F422A4E3043244F304324543039
:1004500043242B24413043242B2443304324413074
:1004600043243D245030432441304324433043242B
:1004700049304324543043244F30432452304324E2
:100480002B24CB2A243076242225861F612A48304B
:1004900069242B242B242B24433043247A304324F7
:1004A0003D3043244C18582AB801B901BA01BB01A8
:1004B0000A23463043242B244F08CE00861B5E2A95
:1004C000CB2A48307624BB254C1CBE2A4808031D85
:1004D000912A4908031D912A4A08031D912A4B08B5
:1004E000031D912A493043244E3043245330432482
:1004F0004530432452304324543043242B2443308A
:1005000043243D247A3043242B24263043242B24B7
:100510005A30432445304324523043244F3043243F
:10052000BD2A4C1DAD2A483076245F258730BF0098
:100530004830C000C101C201222543304324783035
:10054000432425304324433043247A3043243D3030
:1005500043240A232B242B24BD2A43304324783000
:1005600043242D304324433043247A3043243D3008
:1005700043240A23463043242B24CB2A2B242B2428
:100580002B2443304324783043243D3043240A2332
:10059000463043242B24AD28523043244530432495
:1005A0004130432444304324593043242B244C18F5
:1005B000F02A4D304324453043243D244130432428
:1005C0005330432455304324523043244530432490
:1005D0002B246E30CC18E430432420304324092BE4
:1005E0004D304324413043243D2454304324433090
:1005F0004324483043246E30CC18E4304C19253065
:1006000043244D3043244F30432444304324453069
:1006100043240800B91B0E2B2B24102B2D30432410
:10062000CF013808803C03181E2B8430BF002030D7
:10063000C000C101C2015F25CF0A112B8E30BF005F
:100640001C30C0004030C100C20122250D25C1244C
:100650004C08033C031D402B4D08061B4E084F025F
:100660000318402B0310BA0CBB0C0310BA0CBB0CC4
:100670000310BA0CBB0C0310BA0CBB0CCF0A2C2B0A
:100680004F08B800E430B1007030B0003808031DE6
:10069000802B861E742B4C08073C0319742BCC1836
:1006A000742B6E30B1002B243D242B243A08F039F2
:1006B000031D662B2B243A080F39031D622B2B24B4
:1006C0000924F22BBA0E05240924F22B0524052453
:1006D0000924F22B303043243D24582405240524DA
:1006E0000924E430B100F22B303043243D24582457
:1006F00005240524861E7E2B0924F22B2B24F22BA5
:10070000B80B8B2B05243D24582405240924861E70
:10071000F12B0924F22BB80B942B05243D2405243E
:10072000582409240924F22BB80B9D2B05243D24C1
:100730000524092458240924F22B6D30B1006E30B1
:10074000CC1CB000B80BB92B4C08073C0319B32BD9
:10075000861AAC2BCC18B32B05243D245824052431
:1007600009240924F22B05243D2405240924092405
:10077000F12BE430CC18B000B80BD12B4C08073C5F
:10078000031DC52B861BC52B0D2C861A8D2BCC1C4F
:100790008D2B58243D245A2405240524092409249A
:1007A000F22BB80BE52B4C08073C031DDA2B861BFC
:1007B000DA2B0D2C861A962BCC1C962B58243D2414
:1007C0000524052409240924F22B4C08073C031DA9
:1007D000EC2B861BEC2B0D2C2030B100E430B0004C
:1007E000AC2B2B242B244C1CFE2B4C1DFE2B861BD0
:1007F000FE2B253043242B242030032C861E022C74
:100800003108032C300843240800BA0E3A0841246A
:100810000034BB0E3B084124003480303E242B249E
:10082000253043242B244F30432455304324543067
:1008300043242B244F3043243D24463043242B248F
:1008400052304324413043244E3043244730432424
:100850004530432408002030432400343024302421
:100860000730362C4030B3000130372CB301B200D2
:10087000B30B382CB20B382C0034C030C0008601CA
:10088000462C0F393038C00008308600C00E4008B2
:10089000850086148610C00E4008850086148610D8
:1008A0003224003401303E24302428303E24080015
:1008B0002E30432C3030432C84000008B800840ACA
:1008C0000008B900840A0008BA00840A0008BB00C6
:1008D0000800840038088000840A39088000840AEF
:1008E0003A088000840A3B08800008008400000861
:1008F000BF00840A0008C000840A0008C100840AFE
:100900000008C200080084003F088000840A4008F4
:100910008000840A41088000840A420880000800A0
:1009200006086039B400B901BA01BB017030B200E9
:100930009B30B30081019C2C01083B02031CBF2C9F
:10094000031DBA0FA42CB90ABB02B30B9B2CB20B2C
:100950009C2CB2013908031DB22C3A08031DB22C9D
:10096000B21400340608603934020319B92C321469
:100970000034E824383076242225B2010034000007
:10098000A42C3A08C0003B08C10003101030B3008B
:10099000B901BA01BB01C10DC00DBB0DBA0DB90D36
:1009A000B30BD32C00343B308400DD243A30840078
:1009B000DD2439308400DD24CB2C03300007B20065
:1009C000B219800030300007B200B21B8000003442
:1009D0009830B800C301B2013908031D002D3A0850
:1009E000B9003B08BA00BB01B2153908031D002D40
:1009F0003A08B900BA01B2113216390803191D2D8F
:100A00003208B8020310B91B0A2DBB0DBA0DB90D7F
:100A1000B803032DC31FB9130034B9178030B802CF
:100A2000B81F03191D2D3808183CB8000310B90C65
:100A3000BA0CBB0CB80B162D0034B901BA01BB01BE
:100A4000B80100343808031D3F0803191D2D39086B
:100A50004006C3003F08B8078030031C312DB8079B
:100A6000322DB807B917C0170310BC01BD01BE0174
:100A70001830B2003B1C462D4208BE07410803183F
:100A8000410FBD0740080318400FBC07BC0CBD0C4C
:100A9000BE0CB90CBA0CBB0C0310B20B3A2DBC1B2C
:100AA000562DB90DBE0DBD0DBC0DB803C31FBC1333
:100AB0003C08B9003D08BA003E08BB0000343908C4
:100AC0004006C300B917C017B2013908BC003A0884
:100AD000BD003B08BE004208BE024108031C410F96
:100AE000BD024008031C400FBC02BC01BD01BE0199
:100AF000031C812D0310B90CBA0CBB0CBC0C0130CB
:100B0000B2003F08B802031C892D80303207B807B5
:100B10008C2D80303207B8071830B300BE0DBD0DE4
:100B2000BC0DBB0DBA0DB90DB20D4208BB02410898
:100B3000031C410FBA024008031C400FB902400DCC
:100B4000B204321CA52D3E14B02D4208BB0741084B
:100B50000318410FBA0740080318400AB9073E10AE
:100B6000B30B8E2DC31FBC133C08B9003D08BA005F
:100B70003E08BB0000343F08031DC12D4008031987
:100B800000348030C00639084006B20038083F0201
:100B9000031CE22D3F08BE003808BF003E08B80025
:100BA0004008BE003908C0003E08B9004108BE0038
:100BB0003A08C1003E08BA004208BE003B08C20025
:100BC0003E08BB003908C300B917C0174008BC0075
:100BD0004108BD004208BE003F083802BF000319AB
:100BE0000E2E08303F02031C052EBF00BE0D3D082F
:100BF000BE003C08BD00BC0108303F02031C052EAE
:100C0000BF00BE0D3D08BE00BD013F0803190E2EFA
:100C10000310BC0CBD0CBE0CBF0B082EB21F182E4F
:100C2000BC09BD09BE09BE0A0319BD0A0319BC0AE5
:100C30003E08BB073D0803183D0FBA073C080318E0
:100C40003C0FB907B21B2B2E031C0A2DB90CBA0C92
:100C5000BB0CB80A0A2D0318EB2CB909BA09BB0959
:100C6000BB0A0319BA0A0319B90A8030C306EB2C70
:100C7000FF3FFF3FFF3FFF3FFF3FFF3FFF3FFF3F84
:02400E00B23FBF
:00000001FF
